:020000040000FA
:1000000020020010D5000000E5000000E70000001D
:1000100000000000000000000000000000000000E0
:10002000000000000000000000000000E9000000E7
:100030000000000000000000EB000000ED000000E8
:10004000EF000000EF000000EF000000EF000000F4
:10005000EF000000EF000000EF000000EF000000E4
:10006000EF000000EF000000EF000000EF000000D4
:10007000EF00000059060000EF000000EF00000054
:10008000EF000000EF000000EF000000EF000000B4
:10009000EF000000EF000000EF000000EF000000A4
:1000A000EF000000EF000000EF000000EF00000094
:1000B000EF000000EF000000EF000000EF00000084
:1000C0000348854600F006F9004800475507000040
:1000D00020020010064880470648804706488047AF
:1000E00006480047FEE7FEE7FEE7FEE7FEE7FEE71D
:1000F000BD060000CB060000D9010000C1000000D1
:1001000070B54B4D0020696AC905090F0B0000F05E
:1001100053FB1026090B0D0F11131517191B1D1F6B
:100120002123252643481AE0434818E0434816E0B7
:10013000434814E0434812E0434810E043480EE0CF
:1001400043480CE043480AE0434808E0434806E0DF
:10015000434804E0434802E0434800E04348696AFA
:10016000C906890E891C00F011FB314B4033196B15
:100170003F4A89073F4C890F1ED00026012904D031
:1001800002290DD0032921D10CE018688007800FC7
:1001900012D0012810D0022817D0032816D114E05D
:1001A000206013E018688007800F01D00128F2D189
:1001B000A868C005800F01D0226007E0A8682C491C
:1001C000C006C00E401C4843EAE72660996B2068D1
:1001D00000F0DCFA206070BD70B5274A906B2021DA
:1001E00088439063124900230B62184600BF401CED
:1001F000C828FBD30E4801254030056045604360A8
:1002000045604468E407FCD023248C60946B80260E
:10021000B4439463CA68D207FCD0032101634563E9
:1002200043634563416BC907FCD0856370BD000023
:100230000080044020A1070000350C00E0C8100039
:10024000C05C1500006A180040771B0080841E0007
:10025000C0912100009F240040AC2700E03229001B
:1002600020402C00604D2F0000D4300040E13300CE
:10027000001BB70000000010008204401248016813
:1002800040221143016011480268032149020A43D8
:1002900002600F48C26B8A43C263704701220C4957
:1002A00052020028C86B01D0104300E09043C8639D
:1002B00070470122064992020028C86B01D0104302
:1002C00000E09043C8637047808004400080025083
:1002D000C03F0250064C0125064E05E02046E3686B
:1002E00007C82B4398471034B442F7D3FFF7ECFE0E
:1002F000F00700001008000070470000FFFFFFFF3C
:10030000E448016880221143016010214161704777
:1003100070B5E1484168082211434160DE488030F1
:100320000168920311430160DD48DC49006800F078
:100330002DFADC49401E0860D64A01201060106882
:10034000402108431060D848D060002090611368B5
:100350008B431360D54BC9011960CE4BF324014682
:100360004033546290639062D06210635063D063F4
:100370001860586098604D1C1562156A2D04FCD4F5
:10038000491C2029EDD3506010682E2108431060CD
:1003900070BDC04801684908490001607047C44900
:1003A000012008607047BB484068802108407047C2
:1003B00070B5BC4940394A6A096A13040B431F21CE
:1003C000012422468A401A4202D0491EF9D503E090
:1003D000002901DB491C00E00021AE4AF3235362EF
:1003E000037B35241B071B0FE4011B199363437B1D
:1003F00001240525A4036D03002B20D003689BB2C4
:10040000936203686600DB00DB0C9B19D362036810
:100410009BB213630368DB00DB0C1B192B43536394
:100420008388D3639B4BC48840331C6004895C6021
:10043000408998601162106A0004FCD470BD0023EA
:10044000936206687605F60C3419D4621363036868
:100450005B05DB0C5B19E2E730B5924940394A6A2B
:10046000096A13040B431F21012422468A401A42C1
:1004700002D0491EF9D503E0002901DB491C00E048
:100480000021844AB7235362037B13241B071B0FED
:10049000E4011B199363447B05235B03002C18D0F4
:1004A0000468A4B2146304680125E400E40CAD03FD
:1004B00064191C4354638388D363764BC4884033E8
:1004C0001C6004895C6044899C60807B012808D0A2
:1004D00010E00024146304686405E40CE31853631B
:1004E000E9E7506A800880005062506B01235B038B
:1004F000984350631162106A0004FCD430BD024678
:1005000070B50846634980310B681B04FCD47F2317
:100510004B600A600B681B04FCD48B69644D1E059C
:1005200001230024002E10DAF3202B6048608C6138
:100530008C60CC600C614C61CC610C624C628C6252
:100540000A6008680004FCD470BD4A6952044A6914
:1005500006D5D2040E69D20832430260437303E029
:10056000D204520D026044738A691207120F02739B
:10057000CA6982800A6AC2804A6A0281896A4181A4
:100580006B6000F0BAF86C6070BD30B5454A403A17
:10059000536A126A1C041443002201252B4693401F
:1005A000234203D0521C202AF8DB03E0202A01DA80
:1005B000521C00E00022374BF0245C623D4C9C63EF
:1005C0000124E403002910D0C000C00881B2996260
:1005D000000C0443DC621963032189030843586358
:1005E0001A62186A0004FCD430BD400500219962EB
:1005F000C00CD86219632043F1E72A4910B540398D
:100600004A6A096A13040B430021012422468A40E6
:100610001A4203D0491C2029F8DB03E0202901DA23
:10062000491C00E000211B4AF0235362214B9363D5
:1006300000230124E4030028936209D0D4621363E9
:100640000320800350631162106A0004FCD410BDC3
:10065000D36213635463F6E70E490869002817D084
:100660000122D203821A06D04004400C411E1F29E9
:100670000ED8114943E74868020703D54A680823A2
:100680009A434A60C00603D54868102290434860E8
:1006900070470000000005400080044000127A000E
:1006A00000000010800105400123000000E100E08F
:1006B000040000108F1400000C0000102D490020D1
:1006C00000BF401C8842FBDB70472B4801682B4A67
:1006D000114301602A48C16BC908C900C163C16BDD
:1006E00001221143C1632748026802210A430260C4
:1006F0002548C26B8A43C2637047F0B50068FF218A
:10070000024600241225342656270131FF3A85B0CF
:10071000113A0BD10091042168460173447384732C
:100720000571467187717821C1710FE088420FD140
:100730000120FFF7B3FDFF2012300090032168462F
:10074000017344738473057146718771FFF784FEEA
:1007500005B0F0BDFFF792FDFFF7DAFD0020FFF7CF
:100760004CFFFFF716FEFFF71AFE0120FFF7A1FD71
:1007700030BFFDE7A08601008080044040000100FA
:100780004040044000800150C03F015030B50B464E
:10079000014600202022012409E00D46D5409D425B
:1007A00005D31D469540491B2546954040191546E1
:1007B000521E002DF1DC30BD30B47446641E257825
:1007C000641CAB4200D21D46635D5B00E31830BC85
:1007D000184702E008C8121F08C1002AFAD1704762
:1007E000002001E001C1121F002AFBD17047000068
:1007F00010080000000000100C000000D2070000EC
:100800001C0800000C00001014020000E0070000AB
:0C081000006CDC02000000000000000092
:04000005000000C136
:00000001FF
